:100000009F01073083169F0007309C003F3085001A
:10001000FF308600BF3087001C308312A300831698
:100020008717071798011817981618158312980143
:100030009817181718169811013083169900831213
:10004000AD01A401EF106F108C1E242818186F1436
:100050001A08AB006F1C382823082B02031D352813
:1000600098115A30AC00EF1436289815AD012029AC
:1000700000308A002D083D3E82004328B028B52874
:10008000BC28E028E52800308A002B0EAE00AE0C1C
:100090002E0C03394C3E82005028AF28AF287D2813
:1000A00000308A002B0CAE00AE0C2E0C0739593EE6
:1000B000820061287C287C287C287C287C287C285D
:1000C0007C2800308A0007302B05673E82006F28AD
:1000D0007228752878287C287C287C287C28013088
:1000E000AD007C280330AD007C280430AD007C28B6
:1000F00025088A0026088200AF2800308A002B0CD1
:10010000AE00AE0C2E0C0739863E8200AF28AF2819
:10011000AF28AF28AF28AF28AF288E2800308A003C
:1001200007302B05943E8200AF28AF28AF28AF28B8
:100130009C289D28A828AC28AF28EF14AC011C30BF
:1001400024020318A72824082721AC00A40AAF28FA
:10015000A401AC01EF14AF28AC01EF1498152029CD
:100160000230AD002B08A5002029AD012B08A60008
:100170005B30AC00EF142029AD012B08A700270845
:10018000AE00250803178F000313260803178D0000
:1001900083168C170C140000000083120E08031342
:1001A0007521562103170C08031375215621A60A41
:1001B0000319A50AAE0BC1285C30AC00EF1420294E
:1001C0000530AD002B08A9002029AD012B08AA009D
:1001D000290803178E0003132A0803178C00031342
:1001E000250803178F000313260803178D008316B5
:1001F0008C170C1555308D00AA308D008C14000022
:1002000000000C158C170C14000000005F308312E6
:100210000313AC00290803170E0203191229031354
:100220005E30AC0003132A0803170C0203191B29C4
:1002300003135D30AC000313EF14A60A0319A50ADB
:10024000EF1C2629EF142C08752156212228840042
:1002500001308A0004082D3E8200103400341C3422
:10026000013403340E3443346F346E3474347234D6
:100270006F346C346C3465347234323438342D3429
:10028000413407344734723461346D3473346F341D
:100290006E34FF30AF00FF30B0008C1E51291A08B9
:1002A0000800B00B4D29AF0B4B29FC348C1E56298E
:1002B0001A080800A000200E0F3962210F30200517
:1002C00062210034A1000A30210203183730031CD8
:1002D0003030A10721087521003420307521003409
:1002E0000D3075210A3075210034A2000C1E7629CC
:0602F00022089900003411
:02400E003A3F37
:00000001FF
